:100000000C94DE030C9406040C9406040C94060471
:100010000C9406040C9406040C9406040C94060438
:100020000C9406040C9406040C9406040C94060428
:100030000C9406040C9406040C9406040C94060418
:100040000C94650C0C9406040C94D50C0C94AF0C19
:100050000C9406040C9406040C9406040C940604F8
:100060000C9406040C9406044E414E494E495459D2
:10007000494E46CDCCCC3D0AD7233C17B7D1387773
:10008000CC2B329595E6241FB14F0A000020410089
:1000900000C84200401C4620BCBE4CCA1B0E5AAED3
:1000A000C59D742320736368616C746574206B65EF
:1000B000696E656E2041757367616E672061626568
:1000C000722069676E6F72696572742064656E2054
:1000D00045696E67616E6720616E2041352023316E
:1000E000203D204F4E202F202330203D204F4646DC
:1000F0000000000000000000000000000000000000
:1001000000000000000000000000000021206769DE
:1001100062742053656E736F72204944206D697458
:1001200020435243204665686C6572206175732ECA
:100130002045696E65205A61686C206772C3B6C33A
:100140009F65722030207A2E422028213529207385
:100150006368616C74657420C39C626572776163C7
:1001600068756E672065696E2E0000000000000053
:1001700000000000003920676962742056657273C0
:10018000696F6E20617573000000000000000000C0
:10019000000000000000000000000000000000005F
:1001A000000000000000000000000000000000004F
:1001B000000000000000000000000000000000003F
:1001C000000000000000000000000000000000002F
:1001D00000000000000000000000000000003820C7
:1001E0006769627420616C6C652054656D7065721E
:1001F00061747572656E206175732064656D20533E
:1002000070656963686572206D69742053656E73EB
:100210006F726E756D6D6572204120626973207A10
:10022000756D206C65747A74656E20566F726861A6
:100230006E64656E656E2053656E736F72206175B6
:1002400073000000000000372054656D7065726116
:10025000747572756D77616E646C756E6720616C14
:100260006C65722053656E736F72656E20616E737C
:10027000746FC39F656E0000000000000000000066
:10028000000000000000000000000000000000006E
:10029000000000000000000000000000000000005E
:1002A000000000000000000000000000000000004E
:1002B000362050696E737461747573204432206205
:1002C000697320443920756E64204130206269735F
:1002D00020413520616C7320576F726420656D700A
:1002E00066616E67656E000000000000000000009F
:1002F00000000000000000000000000000000000FE
:1003000000000000000000000000000000000000ED
:10031000000000000000000000352054656D70658D
:100320007261747572656E20696D205370656963C2
:1003300068657220616B7475616C6973696572655B
:100340006E0000000000000000000000000000003F
:10035000000000000000000000000000000000009D
:10036000000000000000000000000000000000008D
:10037000000000000000000000000000000000007D
:10038000000034204175746F6D6174697363686532
:10039000732073657269656C6C6573206175736732
:1003A0006562656E206465722054656D706572616A
:1003B000747572656E205B335D206E6163682057D3
:1003C000616E646C756E6720203431204F4E20348E
:1003D00030204F46460000000000000000000000F2
:1003E0000000000000000000000000332053656E94
:1003F000736F72656E204944206D69742054656D79
:100400007065726174757220617573676562656E7F
:1004100000000000000000000000000000000000DC
:1004200000000000000000000000000000000000CC
:1004300000000000000000000000000000000000BC
:1004400000000000000000000000000000000000AC
:1004500000000000322053656E736F72656E204994
:1004600044206D69742050696E20756E6420427559
:1004700073206175736C6573656E2E203231205365
:10048000656E736F72656E2049442065726E657586
:1004900074206175736C6573656E20737065696334
:1004A0006865726E20756E642073657269656C6C28
:1004B00020617573676562656E0000000031204140
:1004C00075746F6D617469736368657320736572A9
:1004D00069656C6C657320617573676562656E2014
:1004E0006465722054656D70657261747572656EB5
:1004F000205B385D206E6163682057616E646C75A7
:100500006E6720203131204F4E203130204F46463B
:1005100000000000000000000000000000000000DB
:10052000000000000000302045696E7374656C6C3B
:10053000756E6720646573204162667261676569E4
:100540006E74657276616C6C73207A2E422E203048
:1005500033303020496E74657276616C6C20616C4A
:100560006C65203330302053656B756E64656E208A
:1005700064656661756C7420333000000000000013
:10058000000000000000000000000000000000610A
:1005900020676962742054656D706572617475724C
:1005A00020766F6E2053656E736F7220284129206C
:1005B0006175732C206220676962742054656D70C8
:1005C00065726174757220766F6E2053656E736FFD
:1005D000722028422920617573202E2E2E207573DB
:1005E0007700000000000000000000000000000094
:1005F000000000000000000041203D2053656E73A4
:100600006F7220494420766F6D20312E2053656E25
:10061000736F72202841292C2042203D2053656EA3
:10062000736F7220494420766F6D20322E205365FF
:100630006E736F7220284229202E2E2E757377201C
:1006400000000000000000000000000000000000AA
:10065000000000000000000000000000000000009A
:10066000003F2041757367616265206465722048B0
:10067000696C66652E20466F6C67656E64204DC39D
:10068000B6676C696368652045696E676162656E0F
:1006900020696E204648454D20756E746572207243
:1006A0006177000000000000000000000000000072
:1006B000000000000000000000000000000000003A
:1006C00000000000000000000000005EBCE2613F8E
:1006D000DD83C29C7E20A3FD1F41009D23BE46DB1F
:1006E00065F88C11AF32CA57E974443A5C417264C0
:1006F00075696E6F5C4E616E6F5C4E616E6F5F31DF
:100700005F776972655F33425F565F312E322E38F4
:100710005C4E616E6F5F315F776972655F33425F18
:10072000565F312E322E382E696E6F204D61792042
:10073000323020323032362032323A33303A3234AC
:10074000006106F8058F052605BD045404EB0382FD
:10075000031903B0024702DE0175010C01A300007A
:10076000000000250028002B0000000000240027C6
:10077000002A0000000000230026002900040404D1
:10078000040404040402020202020203030303033A
:100790000301020408102040800102040810200117
:1007A00002040810200000000800020100000304F9
:1007B00007000000000000000000330D11241FBEE0
:1007C000CFEFD8E0DEBFCDBF25E0AAEFB1E001C09A
:1007D0001D92A230B207E1F711E0A0E0B1E0ECE930
:1007E000F2E302C005900D92AA3FB107D9F713E0DA
:1007F000CEEDD3E004C02197FE010E945417CD3DF9
:10080000D107C9F70E946E0D0C944C190C9400008E
:1008100090E0FC01EB55F84F2491FC01EF56F84FA6
:100820003491FC01E358F84FE491EE23C1F1222307
:1008300039F02330E9F090F4213001F1223011F148
:10084000F0E0EE0FFF1FED58F84FA591B491EC9139
:10085000E32381E090E029F580E008952730A9F0B6
:100860002830C9F0243061F7809180008F7D03C06B
:10087000809180008F7780938000E2CF84B58F775E
:1008800084BDDECF84B58F7DFBCF8091B0008F77A4
:100890008093B000D5CF8091B0008F7DF9CF80E0FC
:1008A00090E00895CF93DF9390E0FC01EF56F84F6E
:1008B00024918358984FFC0184918823C9F090E0DB
:1008C000880F991FFC01E759F84FA591B491FC01DD
:1008D000E15AF84FC591D49161110DC09FB7F894BA
:1008E0008C91209582238C938881282328839FBF15
:1008F000DF91CF910895623051F49FB7F8943C9105
:10090000822F809583238C93E8812E2BEFCF8FB796
:10091000F894EC912E2B2C938FBFEACF3FB7F8942D
:100920008091810290918202A0918302B091840211
:1009300026B5A89B05C02F3F19F00196A11DB11D3A
:100940003FBFBA2FA92F982F8827BC01CD01620F76
:10095000711D811D911D42E0660F771F881F991F31
:100960004A95D1F708958F929F92AF92BF92CF92FE
:10097000DF92EF92FF920E948E044B015C0185E0B2
:10098000C82ED12CE12CF12C0E948E046819790913
:100990008A099B09683E734081059105A8F321E00F
:1009A000C21AD108E108F10888EE880E83E0981E8B
:1009B000A11CB11CC114D104E104F10429F7FF907A
:1009C000EF90DF90CF90BF90AF909F908F90089561
:1009D0002FB7F89460917D0270917E0280917F0222
:1009E000909180022FBF0895AF92BF92CF92DF9275
:1009F000EF92FF920F931F93CF93DF936C017B01D4
:100A00008B01040F151FEB015E01AE18BF08C01764
:100A1000D10759F06991D601ED91FC910190F081D7
:100A2000E02DC6010995892B79F7C501DF91CF919A
:100A30001F910F91FF90EF90DF90CF90BF90AF90FC
:100A40000895FC01538D448D252F30E0842F90E0D4
:100A5000821B930B541710F0CF96089501970895B9
:100A6000FC01918D828D981761F0A28DAE0FBF2F82
:100A7000B11D5D968C91928D9F5F9F73928F90E0D8
:100A800008958FEF9FEF0895FC01918D828D981747
:100A900031F0828DE80FF11D858D90E008958FEF84
:100AA0009FEF0895FC01918D228D892F90E0805C4D
:100AB0009F4F821B91098F739927089585E394E0D6
:100AC0000E94520521E0892B09F420E0822F08952D
:100AD00080E090E0892B29F00E945E0581110C9442
:100AE00000000895FC01A48DA80FB92FB11DA35AD1
:100AF000BF4F2C91848D90E001968F739927848F3E
:100B0000A689B7892C93A089B1898C918370806460
:100B10008C93938D848D981306C00288F389E02D01
:100B200080818F7D80830895EF92FF920F931F93B2
:100B3000CF93DF93EC0181E0888F9B8D8C8D981390
:100B40001AC0E889F989808185FF15C09FB7F8949C
:100B5000EE89FF896083E889F989808183708064E8
:100B600080839FBF81E090E0DF91CF911F910F9133
:100B7000FF90EF900895F62E0B8D10E00F5F1F4F42
:100B80000F731127E02E8C8D8E110CC00FB607FC51
:100B9000FACFE889F989808185FFF5CFCE010E94DF
:100BA0007205F1CFEB8DEC0FFD2FF11DE35AFF4FD6
:100BB000F0829FB7F8940B8FEA89FB89808180626D
:100BC000CFCF682F85E394E00C9494056DE285E324
:100BD00094E00C949405CF93DF93EC01888D8823E7
:100BE000B9F0AA89BB89E889F9898C9185FD03C090
:100BF000808186FD0DC00FB607FCF7CF8C9185FF75
:100C0000F2CF808185FFEDCFCE010E947205E9CF42
:100C1000DF91CF910895DC012C911196ED91FC911B
:100C2000F8948181822B81839281322F3095932396
:100C3000928387E090E00197F1F78181832381839C
:100C400083E290E00197F1F790817894EFECF0E087
:100C50003197F1F7922381E009F480E00895FC01D7
:100C600090810180F281E02D292F209560FF14C032
:100C7000F8948281822382838181892B8183A3E2FC
:100C8000B0E01197F1F78281982B9283789487EDE9
:100C900090E00197F1F70895F8948281822382838E
:100CA0008181892B8183AFEFB0E01197F1F78281C9
:100CB000982B928378948FE090E0EBCFEF92FF92A5
:100CC0000F931F93CF93DF93EC01E62E08E010E023
:100CD000FF24F39461E08E2D8F2109F460E0CE01B2
:100CE0000E942F06FF0C01501109A1F7F894E98129
:100CF000FA8191818881809589238183E981FA81B4
:100D0000928188818095892382837894DF91CF9125
:100D10001F910F91FF90EF900895FC019081018049
:100D2000F281E02DF8948181292F209582238183FF
:100D300078943DE743E050E0315029F1DA01119712
:100D4000F1F780818923C1F3F89482818223828321
:100D50008181892B81837894ABE7B7E01197F1F714
:100D6000F894818182238183A3E1B1E01197F1F7A7
:100D70008081982381E009F080E07894E3E6F6E052
:100D80003197F1F7089580E00895EF92FF920F9365
:100D90001F93CF93DF9310923304DEE087E2E82EB7
:100DA000FF24F394C0913304C330C8F4CD9F800175
:100DB00011240E521B4FC8010E948D06882359F042
:100DC0006CECC8010E945E06C7010197F1F764E46C
:100DD000C8010E945E06CF5FC0933304E3CF0E9438
:100DE000E80460930D0170930E0180930F019093BE
:100DF000100181E080938D028091890290918A0296
:100E0000A0918B02B0918C02809385029093860210
:100E1000A0938702B0938802DF91CF911F910F9129
:100E2000FF90EF9008952F923F924F925F926F92B2
:100E30007F928F929F92AF92BF92CF92DF92EF926A
:100E4000FF920F931F93CF93DF9300D000D0CDB7C5
:100E5000DEB7109234042FE0722E3EE0632E812C18
:100E6000912C40EAA42E42ECB42E50903404809190
:100E70008E02581608F012C1052D10E0709E9001E8
:100E8000719E300D112421573D4F3A83298369010A
:100E900038E0C30ED11CE981FA818085869DC001AE
:100EA00011248E529B4F0E948D06E981FA81E084C5
:100EB000E69C7001112497012E523B4F790165E5A4
:100EC000C9010E945E06E981FA816191FA83E98392
:100ED000C7010E945E0629813A812C153D0599F7CC
:100EE000709EF001719EF00D1124E157FD4FCF016E
:100EF00008969A8389838085869DC00111246EEBB4
:100F00008E529B4F0E945E06109233044090330431
:100F100098E09415C0F4ABEFB1E099E0E0E09150B7
:100F200009F437C08D918E27E82FEF70F0E0E6537B
:100F3000F94F2491E82FE295EF70F0E0E652F94F77
:100F4000E491E227ECCFE981FA81F081F69D9001EE
:100F500011242E523B4F3C832B83E42CF12C98E040
:100F6000C92ED12C312C222423948B819C810E9468
:100F70000B0681113228220C81E0C81AD108A9F78A
:100F8000F701E550FE4F308281E0840D80933304F9
:100F9000BDCF809103028E1360C0709EF001719EE0
:100FA000F00D1124E157FD4F12868081823209F441
:100FB00043C0883209F440C0803109F06FC091E02D
:100FC0009093FA016091FB017091FC018091FA010C
:100FD0008823A9F183E0660F771F8A95E1F7809156
:100FE0000202803149F480910102ECE0F0E0E81B5C
:100FF000F109607F6E0F7F1F709E9001719E300D12
:10100000112421573D4F3A832983072E000C880B6A
:10101000990B0E94A91420E030E040E85DE30E94B3
:101020000815E981FA81638774878587968781E04F
:10103000850D8093340419CF1092FA01C3CF8091AB
:10104000FF01807611F4687FD7CF803211F46C7F76
:10105000D3CF803489F66E7FCFCF709EF001719E22
:10106000F00D1124E157FD4F81858E3F10F48F5F05
:101070008187909100019923D1F2709EF001719EB9
:10108000F00D1124E157FD4F82858F5F828789170C
:1010900070F283869486A586B686C9CF0F900F908E
:1010A0000F900F90DF91CF911F910F91FF90EF90D4
:1010B000DF90CF90BF90AF909F908F907F906F9078
:1010C0005F904F903F902F900895FC010190002079
:1010D000E9F73197AF01481B590BBC0185E394E058
:1010E0000C94F4048F929F92AF92BF920F931F9330
:1010F000CF93DF93CDB7DEB7A1970FB6F894DEBFDD
:101100000FBECDBF19A2423008F44AE08E010F5D38
:101110001F4F842E912CB12CA12CA50194010E946B
:101120003217E62FB901CA01EA30F4F4E05DD801C4
:10113000EE938D01232B242B252B79F790E080E073
:10114000109719F0CD010E946508A1960FB6F8948A
:10115000DEBF0FBECDBFDF91CF911F910F91BF902A
:10116000AF909F908F900895E95CE1CF89E291E084
:101170000C946508CF93DF930E94E105EC010E9477
:10118000B6088C0F9D1FDF91CF910895CF93DF9309
:101190000E946508EC010E94B6088C0F9D1FDF912C
:1011A000CF9108950C9465082F923F924F925F92D1
:1011B0006F927F928F929F92AF92BF92CF92DF9267
:1011C000EF92FF920F931F93CF93DF93109234040B
:1011D000109233048EE0782E9FE0492E80913304E4
:1011E000833008F0ECC0E0903304CE2CD12C7C9CF2
:1011F00080017D9C100D11240E521B4FE8012D968D
:10120000D8011D968C91882301F17C9CF0017D9C76
:10121000F00D1124EE52FB4F138615861486809133
:101220003304789EF0011124EE52FB4F138615868D
:1012300014861286118610861782168215821482F1
:1012400013828F5F80933304C9CFE79C7001112410
:10125000F701EE52FB4F7F0130903404CF010E9422
:101260008D06811108C0D8011B961C921B9718820D
:101270001C961C92D4CF60EFC7010E945E06D1E09D
:10128000612C512CC1E05801BBE0AB0EB11C4801F0
:10129000ECE08E0E911CC7010E940B06282EC701A0
:1012A0000E940B06F1E02F1255C0813009F071C089
:1012B000C13408F4AACF7C9CF0017D9CF00D112470
:1012C000EE52FB4F5386511002C081E085877C9C13
:1012D000F0017D9CF00D1124EE52FB4F8381882399
:1012E00009F493CF349C9001112490E080E0F9013F
:1012F000E80FF91FE157FD4FD701A80FB91F13964B
:101300004C91408301968830910589F7809134048F
:10131000489EF0011124E157FD4F909133049087CE
:1013200011868F5F809334048C3108F45CCFDF9199
:10133000CF911F910F91FF90EF90DF90CF90BF90D2
:10134000AF909F908F907F906F905F904F903F9065
:101350002F900895E62DF0E0281211C0D5018C9150
:10136000C817A8F4D801AE0FBF1F13968C918D2318
:1013700081F4212CC93010F4D401CC935C2EE00F01
:10138000F11F83819D2F9095892383830AC08C133D
:10139000F0CFF801E60DF11D83818D2B838322248C
:1013A0002394622DC7010E942F06CF5FDD0F11F439
:1013B0006394D1E0B7E0B61508F06DCF79CF809196
:1013C000340480938E02B3CFCF93DF93682F70E005
:1013D00090E080E04AE00E947208EC010E94B608AA
:1013E0008C0F9D1FDF91CF9108954F925F926F9266
:1013F0007F928F929F92AF92BF92CF92DF92EF92A5
:10140000FF920F931F93CF936B017C01742EAC015D
:101410009B010E942D17882399F08CE291E0CF91D7
:101420001F910F91FF90EF90DF90CF90BF90AF9002
:101430009F908F907F906F905F904F900C94650875
:1014400046015701E894B7F82FEF3FEF4FE75FE70A
:10145000C501B4010E942D1781110DC02FEF3FEF80
:101460004FE75FE7C501B4010E94A21418161CF4EF
:1014700080E391E0D4CF2FEF3FEF4FE75FE4C70168
:10148000B6010E94281718161CF484E391E0C7CF18
:101490002FEF3FEF4FE75FECC701B6010E94A214A8
:1014A00087FDF3CF20E030E0A901C701B6010E941B
:1014B000A21410E000E087FF08C08DE20E94E10561
:1014C0008C01F7FAF094F7F8F094C0E060E070E077
:1014D00080E09FE37C1641F020E030E040E251E400
:1014E0000E948716CF5FF6CFA70196010E941B16B8
:1014F0002B013C010E94F9164B015C014AE00E945D
:1015000072087C01E00EF11ECC23B1F1C501B401DB
:101510000E94A7149B01AC01C301B2010E941A16DC
:101520004B015C018EE20E94E105E80EF91EC150FC
:1015300018F120E030E040E251E4C501B4010E941E
:1015400008152B013C010E94F9164B01B12CA12C6E
:101550004AE0C501B4010E947208E80EF91EC501F7
:10156000B4010E94A7149B01AC01C301B2010E9407
:101570001A164B015C01DBCFC701CF911F910F9170
:10158000FF90EF90DF90CF90BF90AF909F908F90A3
:101590007F906F905F904F900895CF93DF93C82F07
:1015A00082E00E94E10510923404DFE0809134046F
:1015B00090918E028917E8F48F5B0E94E1058CE31D
:1015C00091E00E94D208E0913404DE9FF0011124E2
:1015D000E157FD4F638574858585968542E00E94BD
:1015E000F5090E94B608809134048F5F809334041B
:1015F000DDCFCC2329F083E0DF91CF910C94BA08A2
:10160000DF91CF91089582E00E94E10588E391E0A7
:101610000E94D208609175027091760290E080E09D
:1016200042E00E9472080E94B60883E00C94BA0857
:10163000CF93DF93882319F082E00E94E105109296
:101640003404DFE09091340480918E02981708F002
:1016500056C08EE391E00E94D20881E491E00E949E
:10166000D2081092330420913304283070F5809111
:101670003404D89FC001112481579D4F820F911DC2
:10168000FC018081803120F483E491E00E94D20843
:101690008091340420913304D89FC00111248157D4
:1016A0009D4F820F911DFC01608170E090E080E011
:1016B00040E10E947208C0913304C73010F40E94C8
:1016C000E605CF5FC0933304CECF8CE391E00E9458
:1016D000D208E0913404DE9FF0011124E157FD4F60
:1016E000638574858585968542E00E94F5090E9490
:1016F000B608809134048F5F80933404A3CF83E0D5
:10170000DF91CF910C94BA081F93CF93DF93D82F1A
:1017100082E00E94E10510923404CFE0809134040D
:1017200090918E02891708F06FC08F5B0E94E105CF
:1017300081E491E00E94D208109233042091330496
:10174000283070F580913404C89FC001112481575E
:101750009D4F820F911DFC018081803120F483E434
:1017600091E00E94D2088091340420913304C89FF4
:10177000C001112481579D4F820F911DFC01608192
:1017800070E090E080E040E10E9472081091330424
:10179000173010F40E94E6051F5F10933304CECF7C
:1017A00085E491E00E94D208E0913404CE9FF001DC
:1017B0001124E157FD4F608570E06F5F7F4F072E6A
:1017C000000C880B990B4AE00E9472088BE491E0B0
:1017D0000E94D208E0913404CE9FF0011124E15719
:1017E000FD4F608570E06F5F7F4F072E000C880B08
:1017F000990B4AE00E9472080E94B6088091340456
:101800008F5F809334048ACF82E591E00E94D208F2
:1018100080918E020E94E409DD2331F083E0DF91A4
:10182000CF911F910C94BA08DF91CF911F91089529
:101830000F931F93CF93DF93EC01888199810097D9
:1018400059F02A813B812617370730F081E0DF917C
:10185000CF911F910F9108958B016F5F7F4F0E9471
:101860007F18009759F0998388831B830A832C8102
:101870003D81232B59F7FC011082E8CF80E0E7CFB0
:10188000CF93DF93EC0162E070E00E94180C288196
:10189000398181110FC02115310519F0C9010E944C
:1018A000F617198218821D821C821B821A82DF9110
:1018B000CF91089582E090E09D838C8364E671E08F
:1018C000C901DF91CF910C9445191F920F920FB669
:1018D0000F9211242F933F938F939F93AF93BF93B6
:1018E00080917D0290917E02A0917F02B091800252
:1018F00030917C0223E0230F2D3758F50196A11D6E
:10190000B11D20937C0280937D0290937E02A09370
:101910007F02B09380028091810290918202A09117
:101920008302B09184020196A11DB11D80938102B2
:1019300090938202A0938302B0938402BF91AF91EF
:101940009F918F913F912F910F900FBE0F901F90FD
:10195000189526E8230F0296A11DB11DD2CF1F9224
:101960000F920FB60F9211242F933F934F935F93D3
:101970006F937F938F939F93AF93BF93EF93FF9357
:1019800085E394E00E947205FF91EF91BF91AF91C2
:101990009F918F917F916F915F914F913F912F9187
:1019A0000F900FBE0F901F9018951F920F920FB6B9
:1019B0000F9211242F938F939F93EF93FF93E091B6
:1019C0004504F09146048081E0914B04F0914C0471
:1019D00082FD1BC0908180914E048F5F8F73209198
:1019E0004F04821741F0E0914E04F0E0EB5CFB4FB6
:1019F000958F80934E04FF91EF919F918F912F913E
:101A00000F900FBE0F901F9018958081F4CF1F93F9
:101A1000CF93DF93EC01162F60E0812F0E945204D8
:101A2000612F70E0FB01EF56F84FE491E883FB0172
:101A3000E358F84FE491F0E0EE0FFF1FED58F84F38
:101A4000859194919A8389831B861D861C861A86AC
:101A5000198618861F821E821D821C821B82DF91BE
:101A6000CF911F910895E5E3F4E01382128288EE8E
:101A700093E0A0E0B0E084839583A683B7838BE1F5
:101A800091E09183808385EC90E09587848784EC56
:101A900090E09787868780EC90E0918B808B81EC3B
:101AA00090E0938B828B82EC90E0958B848B86EC1C
:101AB00090E0978B868B118E128E138E148E6BE0B6
:101AC00082ED94E00E94070D6CE080EE94E00E94AD
:101AD000070D6DE08EEE94E00C94070DCF93DF932D
:101AE000CDB7DEB72A970FB6F894DEBF0FBECDBFD5
:101AF000789484B5826084BD84B5816084BD85B5E9
:101B0000826085BD85B5816085BD80916E008160F4
:101B100080936E001092810080918100826080939A
:101B2000810080918100816080938100809180009C
:101B30008160809380008091B10084608093B100C7
:101B40008091B00081608093B00080917A008460C1
:101B500080937A0080917A00826080937A008091ED
:101B60007A00816080937A0080917A008068809307
:101B70007A001092C10062E082E00E94520462E0AA
:101B800083E00E94520462E084E00E94520462E01A
:101B900085E00E94520462E086E00E94520462E006
:101BA00087E00E94520462E088E00E94520462E0F2
:101BB00089E00E94520462E08AE00E94520462E0DE
:101BC0008EE00E94520462E08FE00E94520462E0C4
:101BD00080E10E94520462E081E10E94520462E0CE
:101BE00082E10E94520462E083E10E945204E0918B
:101BF0004504F091460482E08083E0914104F09135
:101C000042041082E0914304F091440480E1808317
:101C100010924D04E0914904F0914A0486E08083DB
:101C2000E0914704F0914804808180618083E091D5
:101C30004704F0914804808188608083E0914704E4
:101C4000F0914804808180688083E0914704F0919E
:101C5000480480818F7D80830E94C5060E94B30462
:101C60000E94D40880E00E94840B87E691E00E94E5
:101C7000D20883E00E94BA088FE0B82E9FE5292E93
:101C800097E0392E28EE422E23E0522E612C712C43
:101C900030E0832E30E0932EAA24A3940E94B30454
:101CA00020E220930C011092080110920901109279
:101CB0000A0110920B010E94E8046093890270935C
:101CC0008A0280938B0290938C0200910D011091F7
:101CD0000E0120910F0130911001601B710B820BDE
:101CE000930B683E734081059105F0F080918D0261
:101CF0008823D1F080918E028823B1F00E941307CF
:101D000080917B02882329F0809107018A250E9417
:101D1000CD0A80910701882329F080917B028A25D2
:101D20000E94180B10928D028091890290918A0274
:101D3000A0918B02B0918C02409185025091860255
:101D40006091870270918802841B950BA60BB70BDC
:101D500040910301509104016091050170910601C9
:101D600084179507A607B70710F00E94C5060E94C2
:101D7000E804C0907702D0907802E0907902F09069
:101D80007A026C197D098E099F09643671058105F7
:101D9000910508F434C10E94E8046F83788789872D
:101DA0009A870E94E80444E6C40ED11CE11CF11C91
:101DB0002F81388549855A85C20ED31EE41EF51E33
:101DC000C61AD70AE80AF90AC0927702D0927802B6
:101DD000E0927902F0927A0282E00E940804209157
:101DE000750230917602892B09F06AC12160309327
:101DF00076022093750283E00E9408042091750208
:101E000030917602892B09F05DC122603093760211
:101E10002093750284E00E9408042091750230919D
:101E20007602892B09F050C124603093760220930A
:101E3000750285E00E9408042091750230917602B7
:101E4000892B09F043C128603093760220937502F4
:101E500086E00E9408042091750230917602892B59
:101E600009F036C12061309376022093750287E035
:101E70000E9408042091750230917602892B09F0A6
:101E800029C12062309376022093750288E00E9477
:101E900008042091750230917602892B09F01CC14B
:101EA0002064309376022093750289E00E94080432
:101EB0002091750230917602892B09F00FC12068BC
:101EC00030937602209375028AE00E9408042091E4
:101ED000750230917602892B09F002C1316030938E
:101EE0007602209375028EE00E940804209175020C
:101EF00030917602892B09F0F5C03260309376027A
:101F0000209375028FE00E940804209175023091A1
:101F10007602892B09F0E8C0346030937602209372
:101F2000750280E10E9408042091750230917602CA
:101F3000892B09F0DBC0386030937602209375025C
:101F400081E10E9408042091750230917602892B6C
:101F500009F0CEC03061309376022093750282E1A1
:101F60000E9408042091750230917602892B09F0B5
:101F7000C1C03062309376022093750200917502E1
:101F80001091760280917402811158C31F7B1093C7
:101F900076020093750280917202909173029F7B8A
:101FA00090937302809372028091750290917602F1
:101FB0009068909376028093750220910101309190
:101FC00002012F5F3F4F3093020120930101283B14
:101FD0003B4038F4209172023091730282179307CC
:101FE00031F010920201109201010E94030B8091C6
:101FF000750290917602909373028093720285E34A
:1020000094E00E945205181619060CF0C2C085E330
:1020100094E00E94300580930C011A8219821C8280
:102020001B821E821D8266E070E0CE0101960E9436
:10203000180C29813A81811165C02115310519F0EB
:10204000C9010E94F6171A8219821E821D821C8203
:102050001B8285E394E00E9452058C01019759F49C
:1020600085E394E00E9430058E3008F055C0CE0123
:1020700001960E94400C10E000E085E394E00E948D
:102080005205181619067CF485E394E00E94300589
:102090008E3048F090ED980F9A3008F44BC0CE0186
:1020A00001960E94400C85E394E00E9452051816A8
:1020B00019060CF053C085E394E00E943005EFCF81
:1020C0002E7F95CE2D7FA2CE2B7FAFCE277FBCCE8D
:1020D0002F7EC9CE2F7DD6CE2F7BE3CE2F77F0CEAD
:1020E0003E7FFDCE3D7F0ACF3B7F17CF377F24CF8A
:1020F0003F7E31CF3F7D3ECF106410937602009338
:10210000750252CF86E090E09E838D836DE671E08C
:10211000C9010E9445199DCF2D813E81232B21F0BD
:10212000E981FA81309721F410920702E7E0F2E0AA
:102130008083A3CF2D813E810217130720F4E9810C
:10214000FA81309741F410920702E7E0F2E08083D1
:102150000F5F1F4F92CFE00FF11FF9CF89819A8156
:10216000009709F442C00E9426130E94F91660935A
:1021700008017093090180930A0190930B0185E394
:1021800094E00E94EB0589819A81009711F00E94EA
:10219000F617E0910C01E152EF3108F043C20E2E28
:1021A000000CFF0BEA52FF4E0C945417331212131B
:1021B000B912121312131213121312131213121351
:1021C00012131213121312131213F9109711B911DB
:1021D000CB11CF11EA11ED11F011F311F711121318
:1021E00012131213121312130B1260E070E0CB01E2
:1021F000BCCF82E00E94E1052091080130910901E5
:1022000040910A0150910B012F3F8FEF380748078B
:10221000580709F05DC0609103017091040180913D
:10222000050190910601A30192010E943217CA0193
:10223000B9014AE00E94720884E791E00E94C60852
:1022400010910C010FEB010F0A3108F0C5C182E0BB
:102250000E94E10500933404812F0E94E10581E48E
:1022600091E00E94D2081092330420913304283068
:1022700008F0AFC180913404B89EC0011124815789
:102280009D4F820F911DFC018081803120F483E4F9
:1022900091E00E94D2088091340420913304B89ECA
:1022A000C001112481579D4F820F911DFC01608157
:1022B00070E090E080E040E10E94720810913304E9
:1022C000173010F40E94E6051F5F10933304CDCF42
:1022D0002A3031054105510528F1A8EEB3E00E94EE
:1022E000C9156093030170930401809305019093D5
:1022F00006016091030170910401809105019091A4
:102300000601A30192010E943217CA01B9014AE0F5
:102310000E94720884E791E00E94C60883E00E9450
:10232000BA088ECF8EE791E00E94C608E2CF82E025
:102330000E94E1058091080190910901A0910A0194
:10234000B0910B010097A105B10549F410927B02F1
:1023500080917B02882351F087E991E0DDCF0197DE
:10236000A105B105A9F7A0927B02F2CF8AE991E01D
:10237000D3CF8091080190910901A0910A01B091F9
:102380000B010197A105B10511F40E94D40881E069
:102390000E94840B55CF81E00E94180B51CF82E040
:1023A0000E94E1058091080190910901A0910A0124
:1023B000B0910B010097A105B10529F41092070116
:1023C00080910701C7CF0197A105B105C9F7A09278
:1023D0000701F6CF0E94130733CF0E94030B30CFC3
:1023E0000E94C5062DCF81E00E94CD0A29CF82E050
:1023F0000E94E1050AEE16E0F8016491662341F0BF
:1024000085E394E00E9494050F5F1F4F892BA1F78D
:102410000E94B60883CF10928D028091890290911C
:102420008A02A0918B02B0918C02809385029093D6
:102430008602A0938702B093880282E00E94E105A1
:1024400001E417E0F8016591749188E092E00E9440
:102450002A1388E092E00E94C6080E5F1F4F2016E4
:10246000310681F75BCF8091080190910901A0911D
:102470000A01B0910B0185369105A105B10510F453
:102480008093000182E00E94BA0810923404909177
:10249000340480918E02981708F062C08EE391E0B8
:1024A0000E94D20881E491E00E94D2081092330485
:1024B00020913304283070F580913404B89EC00117
:1024C000112481579D4F820F911DFC018081803125
:1024D00020F483E491E00E94D2088091340420919A
:1024E0003304B89EC001112481579D4F820F911D66
:1024F000FC01608170E090E080E040E10E947208A1
:1025000010913304173010F40E94E6051F5F1093FA
:102510003304CECF8EE991E00E94D208E0913404DA
:10252000BE9EF0011124E157FD4F618570E090E0FF
:1025300080E04AE00E9472088BEA91E00E94D20893
:10254000E0913404BE9EF0011124E157FD4F8285D5
:102550000E94E409809134048F5F8093340497CF04
:1025600081EB91E00E94D208809100010E94E40971
:10257000D5CE409108015091090160910A017091F6
:102580000B01423051056105710508F059CE842FC9
:10259000817080937402209175023091760280914F
:1025A000720290917302452B462B472B59F03064F1
:1025B0003093760220937502906490937302809317
:1025C00072023ECE3F7B30937602209375029F7B52
:1025D000F4CF83E00E94BA0810910C010FE9010FBB
:1025E0000A3100F582E00E94E1050093340480EE98
:1025F000810F0E94E1058CE391E00E94D208E091F6
:102600003404BE9EF0011124E157FD4F63857485AB
:102610008585968542E00E94F5090E94B60883E010
:102620000E94BA088114910409F438CB0E945E0517
:10263000882309F431CB0E9400002ECB83E10E9455
:102640000804892B09F458CD1F7B57CD66277727BF
:102650000C943113FB01DC0105900D920020E1F791
:102660000895B0E0A0E0E7E3F3E10C94DA155C0133
:102670007B016115710519F0DB018D939C93850138
:102680000F5F1F4FF501D0818D2F90E00E948114C4
:102690006C01892BB9F5DD32B9F50F5F1F4FD501FC
:1026A0001196DC91C1E05801F1E0AF1AB10843E0A6
:1026B00050E060E770E0C5010E948A14892B69F53B
:1026C000680182E0C80ED11C45E050E06BE670E086
:1026D000C6010E948A14892B21F4680197E0C90E73
:1026E000D11CE114F10419F0D701CD92DC9260E025
:1026F00070E080E89FEFC111FFC060E070E080E80B
:102700009FE7FAC05801BBCFDB3229F485010E5F89
:102710001F4FF501D181C0E0C6CF43E050E068E62D
:1027200070E0C5010E948A14892BE9F0F80110E0DD
:1027300000E020E030E0A9015F01B0ED8B2E8D0EAE
:1027400089E08815C8F19C2E689491F88C2F8870C8
:10275000C2FF16C0811102C00F5F1F4F3196D50115
:10276000DC91C92DE9CFE114F10429F00E5F1F4F70
:10277000F7011183008360E070E080EC9FE7BCC04C
:10278000882311F001501109A5E0B0E00E94C9159D
:102790009B01AC01220F331F441F551F280D311D13
:1027A000411D511D283999E93907490799E1590710
:1027B000A8F2C6609C2ED2CFAEEF8A1206C0C3FD2F
:1027C0003CC09C2E689493F8C9CFDF7DD534A9F521
:1027D00080818D3239F4C061DF011296818162E01F
:1027E00070E006C0DF018B32C1F3119661E070E04A
:1027F00080535D01A61AB70A8A30F8F4E0E8CE16D5
:10280000ECE0DE065CF4B601660F771F660F771FFB
:10281000C60ED71ECC0CDD1CC80ED11C5D01FFEF0F
:10282000AF1ABF0A8C9180538A30A8F1C4FF03C04D
:10283000D194C194D1080C0D1D1DC1FF09C0E11434
:10284000F10431F081E0A81AB108D701AD92BC9231
:10285000CA01B9010E94A714C370C33009F490588B
:102860004B015C0120E030E0A9010E94A214882302
:1028700009F440C0CFE9D0E017FF05C011950195DC
:102880001109C7E8D0E06E01B8E1CB1AD10880E2A7
:10289000E82EF12C0FC0D501B1CFFE012591359165
:1028A000459154910E191F09C501B4010E940815E4
:1028B0004B015C01D501C4010E151F0574F7249767
:1028C000F594E794CC16DD06A9F78A2F880F8B2F95
:1028D000881F8F3F49F020E030E0A901C501B40115
:1028E0000E94A214811106C082E290E09093FD0440
:1028F0008093FC04C501B401CDB7DEB7ECE00C94C5
:10290000F61591110C947515803219F08950855087
:10291000C8F70895FB01DC014150504088F08D91CB
:1029200081341CF08B350CF4805E659161341CF0B1
:102930006B350CF4605E861B611171F3990B089581
:10294000881BFCCF0E94E41408F481E00895E89409
:1029500009C097FB3EF490958095709561957F4FE7
:102960008F4F9F4F9923A9F0F92F96E9BB27939595
:10297000F695879577956795B795F111F8CFFAF4A5
:10298000BB0F11F460FF1BC06F5F7F4F8F4F9F4FD6
:1029900016C0882311F096E911C0772321F09EE834
:1029A000872F762F05C0662371F096E8862F70E09A
:1029B00060E02AF09A95660F771F881FDAF7880F74
:1029C0009695879597F90895990F0008550FAA0BCA
:1029D000E0E8FEEF16161706E807F907C0F0121632
:1029E0001306E407F50798F0621B730B840B950B35
:1029F00039F40A2661F0232B242B252B21F408958A
:102A00000A2609F4A140A6958FEF811D811D089526
:102A10000E941B150C948F150E94811538F00E949E
:102A2000881520F0952311F00C9478150C947E15E0
:102A300011240C94C3150E94A01570F3959FC1F347
:102A4000950F50E0551F629FF001729FBB27F00D5C
:102A5000B11D639FAA27F00DB11DAA1F649F6627B1
:102A6000B00DA11D661F829F2227B00DA11D621F00
:102A7000739FB00DA11D621F839FA00D611D221FBA
:102A8000749F3327A00D611D231F849F600D211D9E
:102A9000822F762F6A2F11249F5750409AF0F1F021
:102AA00088234AF0EE0FFF1FBB1F661F771F881F8A
:102AB00091505040A9F79E3F510580F00C94781535
:102AC0000C94C3155F3FE4F3983ED4F38695779555
:102AD0006795B795F795E7959F5FC1F7FE2B880F30
:102AE000911D9695879597F90895992788270895B8
:102AF00097F99F6780E870E060E008959FEF80ECB1
:102B0000089500240A941616170618060906089553
:102B100000240A9412161306140605060895092EB9
:102B20000394000C11F4882352F0BB0F40F4BF2B28
:102B300011F460FF04C06F5F7F4F8F4F9F4F089568
:102B400057FD9058440F551F59F05F3F71F047955E
:102B5000880F97FB991F61F09F3F79F08795089543
:102B6000121613061406551FF2CF4695F1DF08C062
:102B7000161617061806991FF1CF8695710561057F
:102B800008940895E894BB2766277727CB0197F927
:102B900008950E940B16A59F900DB49F900DA49FC1
:102BA000800D911D112408952F923F924F925F92B4
:102BB0006F927F928F929F92AF92BF92CF92DF924D
:102BC000EF92FF920F931F93CF93DF93CDB7DEB7B2
:102BD000CA1BDB0B0FB6F894DEBF0FBECDBF099446
:102BE0002A88398848885F846E847D848C849B849D
:102BF000AA84B984C884DF80EE80FD800C811B81AB
:102C0000AA81B981CE0FD11D0FB6F894DEBF0FBED9
:102C1000CDBFED010895A29FB001B39FC001A39F56
:102C2000700D811D1124911DB29F700D811D112405
:102C3000911D08955058BB27AA270E9432160C9464
:102C40008F150E94811538F00E94881520F039F404
:102C50009F3F19F426F40C947E150EF4E095E7FBE3
:102C60000C947815E92F0E94A01558F3BA17620743
:102C700073078407950720F079F4A6F50C94C21524
:102C80000EF4E0950B2EBA2FA02D0B01B901900187
:102C90000C01CA01A0011124FF27591B99F0593FCB
:102CA00050F4503E68F11A16F040A22F232F342F13
:102CB0004427585FF3CF469537952795A795F04061
:102CC0005395C9F77EF41F16BA0B620B730B840B76
:102CD000BAF09150A1F0FF0FBB1F661F771F881F2E
:102CE000C2F70EC0BA0F621F731F841F48F4879586
:102CF00077956795B795F7959E3F08F0B0CF939578
:102D0000880F08F09927EE0F9795879508950E94F0
:102D10009B160C948F150E94881558F00E948115FF
:102D200040F029F45F3F29F00C94781551110C9470
:102D3000C3150C947E150E94A01568F39923B1F376
:102D4000552391F3951B550BBB27AA2762177307D1
:102D5000840738F09F5F5F4F220F331F441FAA1F65
:102D6000A9F335D00E2E3AF0E0E832D09150504021
:102D7000E695001CCAF72BD0FE2F29D0660F771FCF
:102D8000881FBB1F261737074807AB07B0E809F0B5
:102D9000BB0B802DBF01FF2793585F4F3AF09E3F3A
:102DA000510578F00C9478150C94C3155F3FE4F34B
:102DB000983ED4F3869577956795B795F7959F5F7D
:102DC000C9F7880F911D9695879597F90895E1E0C9
:102DD000660F771F881FBB1F621773078407BA0728
:102DE00020F0621B730B840BBA0BEE1F88F7E09583
:102DF00008950E94A81588F09F5798F0B92F992739
:102E0000B751B0F0E1F0660F771F881F991F1AF0D5
:102E1000BA95C9F714C0B13091F00E94C215B1E063
:102E200008950C94C215672F782F8827B85F39F062
:102E3000B93FCCF3869577956795B395D9F73EF46E
:102E400090958095709561957F4F8F4F9F4F089516
:102E50000E94E41408F48FEF08950E94E414880B94
:102E6000990B0895A1E21A2EAA1BBB1BFD010DC0F0
:102E7000AA1FBB1FEE1FFF1FA217B307E407F5072A
:102E800020F0A21BB30BE40BF50B661F771F881F06
:102E9000991F1A9469F760957095809590959B019C
:102EA000AC01BD01CF010895EE0FFF1F0590F49115
:102EB000E02D09940F931F93CF93DF9382309105F8
:102EC00010F482E090E0E0910005F091010530E01F
:102ED00020E0B0E0A0E0309799F42115310509F425
:102EE0004AC0281B390B24303105D8F58A819B81D3
:102EF0006115710589F1FB0193838283FE0111C085
:102F0000408151810281138148175907E0F0481729
:102F1000590799F4109761F012960C931297139633
:102F20001C933296CF01DF91CF911F910F9108959D
:102F30000093000510930105F4CF2115310551F0E0
:102F40004217530738F0A901DB019A01BD01DF01E7
:102F5000F801C1CFEF01F9CF9093010580930005EF
:102F6000CDCFFE01E20FF31F8193919322503109DF
:102F700039832883D7CF2091FE043091FF04232B7F
:102F800041F420911301309114013093FF042093F8
:102F9000FE0420911101309112012115310541F4F7
:102FA0002DB73EB74091150150911601241B350BEA
:102FB000E091FE04F091FF04E217F307A0F42E1B4A
:102FC0003F0B2817390778F0AC014E5F5F4F24178D
:102FD000350748F04E0F5F1F5093FF044093FE04E7
:102FE000819391939FCFF0E0E0E09CCFCF93DF936C
:102FF0000097E9F0FC01329713821282A09100053C
:10300000B0910105ED0130E020E01097A1F420819E
:103010003181820F931F2091FE043091FF04281705
:10302000390709F061C0F093FF04E093FE04DF91DB
:10303000CF910895EA01CE17DF07E8F54A815B8159
:103040009E0141155105B1F7E901FB83EA834991DE
:103050005991C40FD51FEC17FD0761F48081918150
:103060000296840F951FE901998388838281938159
:103070009B838A83F0E0E0E012968D919C911397F8
:103080000097B9F52D913C911197CD010296820FD1
:10309000931F2091FE043091FF042817390739F659
:1030A000309751F51092010510920005B093FF047E
:1030B000A093FE04BCCFD383C28340815181840F8F
:1030C000951FC817D90761F44E5F5F4F88819981BA
:1030D000480F591F518340838A819B819383828348
:1030E0002115310509F0B0CFF0930105E0930005FB
:1030F0009ECFFD01DC01C0CF13821282D7CFB0E09A
:10310000A0E0E5E8F8E10C94D6158C01009751F4A5
:10311000CB010E945A178C01C801CDB7DEB7E0E1A0
:103120000C94F215FC01E60FF71F9C0122503109A7
:10313000E217F30708F49DC0D901CD91DC911197F6
:10314000C617D70798F0C530D10530F3CE010497E4
:103150008617970708F3C61BD70B2297C193D19305
:103160006D937C93CF010E94F617D6CF5B01AC1A0A
:10317000BD0A4C018C0E9D1EA0910005B091010569
:10318000512C412CF12CE12C109731F58091FE044B
:103190009091FF048815990509F05CC04616570602
:1031A00008F058C08091110190911201009741F4EC
:1031B0008DB79EB74091150150911601841B950B58
:1031C000E817F90708F055C0F093FF04E093FE04F8
:1031D000F90171836083A0CF8D919C911197129614
:1031E0006C90129713967C901397A815B90559F512
:1031F0006C0142E0C40ED11CCA14DB0420F1AC0106
:103200004A195B09DA011296159780F0628273827F
:1032100051834083D9016D937C93E114F10471F0E3
:10322000D7011396FC93EE93129776CF22968C0FCC
:103230009D1FF90191838083F301EFCFF093010586
:10324000E093000569CF4816590608F42C017D016A
:10325000D3019ACFCB010E945A177C01009749F005
:10326000AE01B8010E943C19C8010E94F6178701FF
:1032700053CF10E000E050CFFB01DC0102C0019011
:103280000D9241505040D8F70895FB01DC010190A8
:0C3290000D920020E1F70895F894FFCFA4
:10329C0007B80B3075000001FFFFFFFF20307500F1
:1032AC0000000002058000000000009405F40421D9
:1032BC0005EB055205300544050D0A006E616E00E4
:1032CC00696E66006F76660050696E733D00494406
:1032DC00003A0030002042757320002050696E20A7
:1032EC003100416E7A61686C2053656E736F726544
:1032FC006E3A20002D310052656164790020202047
:10330C00202020002053656B756E64656E00313093
:10331C002053656B756E64656E2073696E64206DE9
:10332C00696E696D756D004F4E004F464600204327
:10333C0052435F676573616D747C00204352437C1C
:10334C00005365747A652054656D7065726174758F
:10335C007220617566202D38302E30206265692010
:10336C00416E7A61686C2061756665696E616E6428
:10337C006572666F6C67656E6465204352432046C8
:0A338C0065686C6572203E3D20006C
:00000001FF
